:10000000412883169B0083161C141A089B0A3D285E
:1000100083169A001C1555309D00AA309D009C1433
:100020009C1810281C119B0A3D288001840AFF3E61
:10003000031D15283D28A401A300FF30A307031CBE
:10004000A407031C3D280330A200DF3029201D280F
:10005000A201E83EA100A209FC30031C3228A1073E
:1000600003182F28A1070000A20F2F2821183828D5
:10007000A11C3C2800003C280800831383120313B2
:100080000800FF2383169000831207309900850132
:1000900087010830831685008701203084004030B6
:1000A0008312152064301B207A2085160130A400AD
:1000B00090301C200130AA0085195F28AB14013054
:1000C000A200F4302920AA0A031D5C288512AB1C6B
:1000D00079280130AA000A302A0203187828203033
:1000E00085060130A400F4301C20AA0A031D6B28E9
:1000F000AE20C828051205108510051107108710BD
:100100000711871107128712AB188728851208007C
:100110008310851983148318AB15831CAB11AA01B6
:1001200003018519013EAB19013C03190130031D80
:100130000301A50032302A02013003180301A5058E
:100140000319A428AA0A902832302A02031DA928DC
:100150002B140330A200E830292008000130A7004A
:100160002C30A600A608031DB828A7080319C72825
:10017000A603260A0319A7038519C2280130A70080
:100180002C30A6000130A200F4302920B22808004B
:100190007A20851DCC28C928AA01013085190301C0
:1001A000A50034302A02013003180301A505031904
:1001B000DB28AA0ACD2834302A020318E028C828F0
:1001C00085160230A2005830292088200301AB1D7B
:1001D000013E03192813031D281788202B15AB1D7A
:1001E0002B1188202916AB1D29128820A915AB1DBB
:1001F000A91188202915AB1D29118820A914AB1D30
:10020000A91088202914AB1D29108820A816AB1D21
:10021000A81288202816AB1D28128820A815AB1D0F
:10022000A81188202815AB1D28118820A814AB1D03
:10023000A81088202814AB1D28102B1C21292B1056
:10024000C828AB1C2429692900300120A0002908F6
:100250002002031D6829A808031D302905166729F7
:1002600001302802031D36290514672902302802AF
:10027000031D3C298514672903302802031D4229E8
:100280000515672904302802031D4829071467292A
:1002900005302802031D4E298714672906302802DD
:1002A000031D54290715672907302802031D5A2901
:1002B0008715672908302802031D6029071667295A
:1002C00009302802031D662987166729C828AE2031
:1002D000C82883169B01831229080820AB1001301F
:1002E000AA0015302A0203187C2920308506963092
:0E02F0001B20AA0A031D7129AE20C8287E29F2
:02400E00043E6E
:024200000000BC
:00000001FF
